:020000040800F2
:10000000B00E00209D01000873300008172B000877
:1000100071300008DF0900081141000800000000ED
:1000200000000000000000000000000099370008F8
:10003000830A0008000000002B360008ED37000896
:10004000B7010008B7010008B7010008B7010008B0
:10005000B7010008B7010008850A0008D10A0008A6
:10006000310B0008B7010008B7010008E1090008DA
:10007000B7010008B7010008B7010008B701000880
:10008000B7010008B701000881080008B70100089F
:10009000B7010008B7010008B7010008B701000860
:1000A000B7010008B7010008B7010008B701000850
:1000B00081380008B701000800000000B7010008FF
:1000C000B70100080000000000000000B7010008B0
:1000D00000000000B7010008B7010008B7010008E0
:1000E000B7010008B7010008000000000000000090
:1000F0000000000000000000000000000000000000
:1001000000000000000000000000000000000000EF
:100110000000000000000000B7010008B70100085F
:1001200000000000000000000000000000000000CF
:1001300000000000000000000000000000000000BF
:10014000B7010008B701000800000000B70100086F
:10015000B7010008B7010008B7010008B70100089F
:10016000B7010008B701000800000000000000000F
:10017000000000000000000000000000000000007F
:1001800000000000B7010008DFF80CD000F02EFBE3
:100190000048004719410008B00E0020064880477B
:1001A00006480047FEE7FEE7FEE7FEE7FEE7FEE75C
:1001B000FEE7FEE7FEE7FEE7713800088901000868
:1001C000202A04DB203A21FA02F00021704721FAAC
:1001D00002F3D040C2F12002914008431946704713
:1001E00010B5431A934209D28318881803E010F817
:1001F000011D03F8011D521EF9D210BD40EA010392
:100200009B0703D009E008C9121F08C0042AFAD2CC
:1002100003E011F8013B00F8013B521EF9D210BD7A
:10022000D2B201E000F8012B491EFBD27047002238
:10023000F6E710B513460A4604461946FFF7F0FFE5
:10024000204610BD421C10F8011B0029FBD1801A6A
:1002500070472DE9FE4F804681EA0300C00F0C462F
:10026000009021F0004123F00045B8EB0200A941C5
:1002700005D24046214690461C460B46024623F0D6
:100280000040104347D0270DC7F30A00C3F30A51BB
:100290000290401A019040286BDAC3F3130040F437
:1002A000801B0098924620B10023D2EB030A63EB37
:1002B0000B0B01985946C0F14002504600F058F926
:1002C00006460D4650465946019A00F060F910EB7B
:1002D00008006141002487EA115284EAE7731A4357
:1002E00040D0009A62B3019A012A4FEA075215DC06
:1002F000001B61EB02014FF0004202EA0752CDE918
:100300000042001C41F5801132462B4600F07EF978
:1003100003B0BDE8F08F40462146F9E7001B61EBD2
:100320000201001C41F5801300185B412018A2F562
:10033000001747EB030140EAD570B6196D4111E093
:100340006D084FEA360645EAC0754FEA0752001BB2
:1003500061EB0201001C41F5801149084FEA3000B1
:100360000019514132462B4603B0BDE8F04F00F072
:100370003EB90098012240000023D0EB020263EB5B
:10038000E073009821464FEAE074B8EB000061EB9F
:100390000401E9E783F000435BE781F0004158E79F
:1003A0002DE9F04D81EA030404F0004B21F00045F3
:1003B00014464FF0000A23F0004150EA050220D015
:1003C00054EA01021DD0C5F30A570246C5F31303D0
:1003D000C1F31300C1F30A5640F4801543F48013AF
:1003E000A7EB0608101BD64608F2FD3873EB050094
:1003F00002D308F1010801E092185B41B8F1000F47
:1004000003DA00200146BDE8F08D00204FF4801192
:10041000064684460EE0171B73EB050705D3121B37
:1004200063EB050306434CEA010C49084FEA300030
:1004300092185B4150EA0107EDD152EA030012D055
:1004400082EA040083EA0501084305D0101BAB4192
:1004500006D20122002306E000224FF0004302E012
:100460006FF0010253101AEB06004CEB085110EB31
:100470000A0041EB0B01BDE8F04D00F0B8B870B5D3
:10048000C1F30A5201F000450024C1F3130140F208
:10049000FF3341F480119A4201DA002070BD40F22E
:1004A00033439A42A2F2334203DC5242FFF788FE02
:1004B00000E090402C43F1D0404270BD00F000427B
:1004C00030F000400AD0C10D01F56071C0F3160094
:1004D00042EA0151C208400711437047002001461B
:1004E000704730B50B46014600202022012409E068
:1004F00021FA02F59D4205D303FA02F5491B04FADD
:1005000002F52844151EA2F10102F1DC30BD2DE9EF
:10051000F05F0546002092469B4688460646814687
:1005200040241BE02846414647462246FFF748FE46
:1005300053465A46C01A914110D3114618462246D6
:1005400000F016F82D1A67EB01084F4622460120ED
:10055000002100F00DF817EB00094E41201EA4F118
:100560000104DFDC484631462A464346BDE8F09F99
:10057000202A04DB203A00FA02F100207047914063
:10058000C2F1200320FA03F3194390407047202A58
:1005900006DBCB17203A41FA02F043EAE07306E0AB
:1005A00041FA02F3D040C2F12002914008431946BB
:1005B000704710B541000CD0C0F3C751962908DC34
:1005C0007E2909DC06DB410204D000F0004040F047
:1005D0007E5010BD002010BDC1F19604C4F1200171
:1005E00000FA01F1E04000F013F9A04010BD10B591
:1005F000141E73F1000408DA401C41F10001921846
:100600005B411A4301D120F0010010BD2DE9F04DEE
:1006100092469B4611B1B1FA81F202E0B0FA80F243
:1006200020329046FFF7A4FF04460F4640EA0A0036
:1006300041EA0B0153465A46084313D0114653EA88
:10064000010019D0C8F140025046FFF7B9FD054638
:100650000E46504659464246FFF78AFF084305D0EA
:10066000012004E020463946BDE8F08D0020054316
:1006700046EAE0762C4337430A986305E40AA0EB88
:1006800008000022FD0A44EA47540A3002D500203F
:100690000146E9E7010510196941DDE9084500193E
:1006A0006941BDE8F04DA2E72DE9FE4F81EA030460
:1006B00004F0004421F0004100944FF0000B23F0BF
:1006C000004350EA01045ED052EA03045BD0C3F356
:1006D0000A54C1F30A552C44A4F2F3340194A0FB4C
:1006E0000254C1F3130141F48011C3F3130343F423
:1006F000801301FB024400FB034E840A970A44EA7C
:10070000815447EA8357A4FB076802958D0A05FBCD
:1007100007854FEA932C04FB0C542705029D4FEAF2
:10072000065847EA1637B5EB08056EEB070C870E3F
:10073000920E47EA811742EA8312A7FB0201B6EB49
:100740000B0164EB00042B0D43EA0C335E1844EB01
:100750001C50DA465146E7FB0201C5F313044FEA89
:100760000B3343EA14534FEA0432019C43EA060375
:10077000A4F10C040294009CCDE900B4FFF746FFFD
:1007800003B0BDE8F08F00200146F9E7C1F30A523B
:10079000C1F3130140F2FF3341F480119A4202DAAF
:1007A00000200146704740F233439A42A2F233429E
:1007B00002DC5242FFF704BDFFF7DABE30B5041E7B
:1007C00071F1000404DB4FF00044404264EB01018E
:1007D000141E73F1000405DB1C464FF00043524227
:1007E00063EB0403994208BF904230BD064C074DAD
:1007F00006E0E06840F0010394E8070098471034F1
:10080000AC42F6D3FFF7C4FC0C6400082C6400086B
:100810000029A8BF7047401C490008BF20F0010014
:10082000704710B4B0FA80FC00FA0CF050EA0104F2
:1008300004BF10BC704749B1CCF1200421FA04F484
:1008400011FA0CF118BF012121430843A3EB0C015D
:10085000CB1D4FEA00614FEA102042BF002010BCC0
:10086000704700EBC35010440029A4BF10BC704770
:10087000401C490008BF20F0010010BC7047000078
:10088000014800F045BB00BF4C0600200146406A0D
:10089000026C12F0500F03D0806B026B08461047B9
:1008A0000168026C42F400720264C96811F4406F7E
:1008B00001D000F029BB417E0029FAD1016C21F45E
:1008C00080710164016CC904F3D4016C41F0010131
:1008D000016400F019BB406A016C41F04001016401
:1008E000416C41F00401416400F010BB406A00F02B
:1008F0000CBBB0B50446006802F066FC02D101688A
:10090000C90701D10020B0BD816801F00D010129A6
:1009100015D1816841F0020181600321016000F07E
:1009200067FF054620688068C007EBD000F060FFD5
:10093000401B0328F6D320688068C007F2D002F07D
:1009400043BE0000B0B50446006802F03DFC02D191
:100950000168C9071AD181680D4A114201D002F01D
:1009600033BE816841F00101816000F041FF05461E
:1009700020680068C00709D100F03AFF401B032837
:10098000F6D320680068C007F2D1E8E70020B0BDC8
:100990003F00008070B5044603F0CEFE0026F0B2A2
:1009A000A042A8BF70BD0125280607D0E8B203F019
:1009B000D9FE0A2000F028FE6D00F5E78020010630
:1009C00008D0C5B2284603F0CDFE0A2000F01CFE78
:1009D0006808F4E7002003F0C5FE0136DFE7FEE714
:1009E0004E48016989BB416949B31949194A0988C7
:1009F00090ED060A92ED011A92ED003A028802EE9D
:100A0000101A04EE102AB8EE422AB8EE444A23EE39
:100A1000023A04EE013A30EE030A80ED060A018044
:100A200090ED070A90ED091A90ED083A23EE022A9C
:100A300004EE012A30EE020A80ED070A05E00449BF
:100A400009880180416901314161034800F030BDEE
:100A5000BC040020040000209C060020F0B5D0E972
:100A60000045D0E90F60012707FA00F0102D7060F3
:100A70000846636008BF1046A06008BF0A46E260EF
:100A8000F0BD704770B5254CA06801280ED098B90C
:100A90002348142202F032FB0120012602F07EFEE0
:100AA0002048068020482561056005E01F4801F0C8
:100AB0001DFD1C4801210180A068411C0028C8BF01
:100AC0000021A1600120BDE8704000F0B1BD00BF71
:100AD000B0B5124CE068012817D090B910483C22FC
:100AE00002F00CFB0F48042101800F48656005608F
:100AF0000120012502F052FE0C48256101F0F6FCB0
:100B0000E068012803DA013002E0002020610020C3
:100B1000E0600220BDE8B04000F08ABD7C0000200B
:100B2000900700202000002024000020DC07002087
:100B3000042000F07DBDEFF3108072B6FEE7704731
:100B40007047704770470000F0B590F83C20012ACC
:100B500001D1022162E003689A68520737D4E74A5C
:100B6000B3F1A04F144608BF04F5807425686D07E3
:100B70002DD40D68D2F8006326F4604655B34F6853
:100B80003E4390F8307046EA4736C2F800639E68EC
:100B900006F00306012E02D11E68F6073AD124683A
:100BA00004F00304012C09D14FF0A044B3F1A04F8D
:100BB00008BF02F1F8042368DB072BD1D2F8003319
:100BC000896840F61F74A3432943194320E002F0CB
:100BD000F1FA20E0C2F80063996801F003010129ED
:100BE00002D11968C90715D1216801F00301012953
:100BF00009D14FF0A041B3F1A04F08BF02F1F801B5
:100C00000968C90706D1D2F8001340F61F7399434B
:100C1000C2F800130021002280F83C200846F0BDF5
:100C2000F8B50022009290F83C20012A01D102215F
:100C300060E1012280F83C20026893685B0700F1C4
:100C4000FC804C68042C0FD804EB4404D1F800C09D
:100C50001F2664000CFA04F506FA04F4166B26EA63
:100C600004042C43146324E0092C0BD804EB440344
:100C70006FF01D0402F024FC566B26EA04042C439A
:100C8000546316E004EB44030E2C09D86FF03B04C8
:100C900002F016FC966B26EA04042C43946308E0E9
:100CA0006FF0590402F00CFCD66B26EA04042C43C6
:100CB000D463946814F00C0F24D0936803F00303FA
:100CC000012B03D11368DB0740F01081012303FAE5
:100CD0000CF4CB68012B41D1D2F8B0302343BCF1E6
:100CE0000A0FC2F8B03050D30CEB4C0389680724CC
:100CF0001B3B994004FA03F3946924EA0303194364
:100D0000916130E00CEB4C04BCF1090F4FF014057D
:100D100088BF1E3C88BF1825072356598F68A340FB
:100D2000A74026EA03033B435351D5680B695C1E79
:100D3000032C00F29080062303EA95034D699D4041
:100D4000DFE804F002B0BAC445EA8C63146E6A4D61
:100D50002C40234343F000431366AEE7D2F8B010B3
:100D6000A143C2F8B010BCF1120F22D0BCF1110F98
:100D700024D0BCF1100F40F0B9806049D1F80013C5
:100D8000090200F1B380012120E00CEB4C038968DB
:100D900007240333994004FA03F3546924EA030354
:100DA0001943BCF1110F516108D0BCF1120F40F092
:100DB0009D805249D1F80013490203E04F49D1F810
:100DC0000013C9014FF0000100F19180936803F016
:100DD0000303012B02D11368DB072ED1474CB2F17C
:100DE000A04F234608BF03F580731B6803F003037D
:100DF000012B09D14FF0A043B2F1A04F08BF04F17D
:100E0000F8031B68DB0718D1D1B1B2F1A04F6DD147
:100E1000D4F800133B4A41F40001C4F800133849E8
:100E20000968B1FBF2F101EB8101490000910099E1
:100E300000295BD000990139F8E702F0BBF956E0D0
:100E4000BCF1110F4CD1B2F1A04F4FD1D4F8001327
:100E500041F0807148E0136E4FEA8C6403F0F84370
:100E6000A34203D1136E23F000431366536E03F0C5
:100E7000F843A34203D1536E23F000435366936EAD
:100E800003F0F843A34203D1936E23F0004393662B
:100E9000D36E03F0F843A3427FF40FAFD36E23F079
:100EA00000431BE045EA8C63546E134D2C402343F2
:100EB00043F00043536600E745EA8C63946E0E4DA1
:100EC0002C40234343F000439366F6E645EA8C63E7
:100ED000D46E094D2C40234343F00043D366ECE627
:100EE000D4F8001341F48001C4F80013002100225B
:100EF00080F83C200846F8BD00F0FF0308000050D1
:100F00001C00002040420F007047704770470000EF
:100F1000B0B5044600688E4D0168490702D54168A6
:100F2000490705D40168090740D5416809073DD53F
:100F3000214651F8402FD20603D40A6842F40072C9
:100F40000A602A68D2060DD02A6802F01F02052A1C
:100F500008D02A6802F01F02092A18BFB0F1A04F7A
:100F600040F0E58000F10C02126802F06EF917D132
:100F70000268120714D5826852070BD4426822F027
:100F80000C024260086820F4807008600868C004A1
:100F900002D505E002F0B3F9086840F001000860EE
:100FA0002046FFF7B1FF20680C2101600168890627
:100FB00002D54168890605D40168490626D54168ED
:100FC000490623D5214651F8402F42F400520A60C9
:100FD0002A68D2060DD02A6802F01F02052A08D01E
:100FE0002A6802F01F02092A18BFB0F1A04F40F092
:100FF000A18000F10C021268C36C13F0C00F64D022
:101000002046FFF79CFD2068602101600168090609
:101010000CD54168090609D5206C40F48030206465
:10102000204600F07BF92068802101600168C90535
:101030000DD54168C9050AD5206C40F40030206404
:101040002046FFF77EFD20684FF480710160016843
:1010500089050DD5416889050AD5206C40F48020AA
:1010600020642046FFF76EFD20684FF40071016098
:101070000168C9061AD54168C90617D5616B0129EF
:1010800006D02968C9064ED0296811F4404F0BD00C
:10109000206C40F480602064606C40F0020060646A
:1010A0002046FFF733FF20681021016001684905E1
:1010B00002D54168490500D4B0BD02F05DF8016079
:1010C0002046BDE8B040FFF73BBD930102D502F0DA
:1010D000BCF895D10268520692D52A68D2060CD087
:1010E0002A6802F01F02062A07D02A6802F01F02AF
:1010F000072A18BFB0F1A04F26D100F10C021268E8
:1011000092023FF57DAF8268120716D4426822F042
:1011100060024260086820F4805008600868C005DA
:101120003FF56EAF0BE0C168C907B1D1BCE7A5F5CB
:101130003F7219E7A5F53F725DE702F0E0F8086835
:1011400040F0010008605BE7A5F53F72D7E700BFFC
:1011500008030050BCB5044600200190B4B3206CD5
:10116000C00635D4206C0025A8BB20466564C4E9C0
:10117000125584F83C5000F0D3F820688068C00015
:1011800029D402F026F90546206C00F0100028430F
:1011900021D12068216C41F2021291430231216475
:1011A000816821F040518160816841F08051816007
:1011B000554856490068B0FBF1F000EB8000400054
:1011C0000190019830B101980138F9E70120BCBDC8
:1011D000002512E0002520688168C90002D58068DA
:1011E00080000AD5206C012540F0100020F002009C
:1011F0002064606C40F001006064206C00F010001E
:10120000284348D120688168490744D4216C21F4DF
:1012100081710231216401F0D7FF02D10168C90751
:101220001DD13B49B0F1A04F0A4608BF02F58072BC
:10123000126802F00302012A09D14FF0A042B0F176
:10124000A04F08BF01F1F8021268D20707D1626807
:10125000D1F8003323F440331A43C1F80023627EEF
:10126000616B530303F58053012908BF5303D4E98D
:1012700002152943194394F82030012B15D17AB176
:10128000226C42F0200222F002022264626C42F0E0
:101290000102626409E0012010216FF012022EE0C9
:1012A000626A1C4B03EB42421143A26A012A02D03C
:1012B0001143E26A1143826812F00C0F0BD1C2682D
:1012C00044F202039A43C260227E94F8303041EA2D
:1012D000823141EA4301C2680F4B1A401143C16099
:1012E000016B226921F00F01012A02D1E269013A62
:1012F00011430163002001216FF003026064236C3D
:101300001A4011432164BCBD1C00002040420F0064
:10131000080000500000FFFF07C0F0FF704700000A
:1013200070B586B0044600680026CDE90466B0F1C9
:10133000A04F3AD11E48016841F080510160016818
:1013400001F0805100910099016841F40021016091
:10135000006800F400200090032003960290012012
:101360000190009801A9134800F06CF9124D134B3D
:101370004FF480604FF480718022C5E90410284644
:10138000C5E90036C5E90262C5E9066600F0D6F88F
:1013900008B1FFF7D0FB1220002100226C62A56388
:1013A00000F0AEFB122000F09FFB06B070BD00BF46
:1013B00014100240000800489C060020080002406B
:1013C0002DE9F04101F0BFFF02D401F0E9FE01D1A7
:1013D000022714E00120324D84F83C00D5F8FC02CD
:1013E000C00602D00020012707E0204690460E46A6
:1013F000FFF7A8FA30B10746002084F83C003846D1
:10140000BDE8F08101F065FF00F580702064D5F83B
:10141000FC02C00611D02168B1F1A04F0DD0206CA4
:1014200040F48010206405F1F400814212D155F897
:10143000F40B8001294608D40CE02168206C20F4CC
:1014400080102064C868800104D5206C012262F3FA
:101450000D302064206C134A134B144D0027C00438
:101460004FF0000044BF606C20F0060060641C2058
:101470000860486840F01000486084F83C70A06B39
:10148000C0E90A5302634346CA6842F00102CA60D7
:101490004031324600F084F8206801F0A4FEAEE747
:1014A0000C000050D7080008ED0800088D0800085F
:1014B000F0B5D0E90F13026804240E6804FA03F5AE
:1014C0001468354201D0670719D402259D40354282
:1014D00001D0A7071DD426FA03F52D072CD5240724
:1014E0002AD5146824F00E041460012202FA03F3D2
:1014F0004B604FF4807101848263016B18E01368C4
:101500009B0603D4136823F0040313604D60C16A83
:101510000EE013689B0606D4012380F8213013687F
:1015200023F00A031360002280F820204D60816AB6
:1015300011B1BDE8F0400847F0BD000048B32DE907
:10154000F041D0E9001E00F1100CD0E9028443F60E
:10155000F0739CE8E0100A689A434FF4807342EA03
:101560000E0242EA080222432A4332433A4342EA45
:101570000C020A600384094B074A19441423B1FB87
:10158000F3F18900C0E90F2100218163BDE8F0413A
:1015900000E001210846704700000240F8FFFDBF4F
:1015A000B0B5044690F8200001281DD0012084F831
:1015B000200094F82100012813D10020A06302200C
:1015C00084F821002068056825F0010505602046A3
:1015D000FFF744FA2068E26A01683AB141F00E016F
:1015E0000AE0002084F820000220B0BD41F00A018A
:1015F0000160016821F004010160016841F001010E
:1016000001600020B0BD0000B0B5044600F0F0F865
:1016100005460548611C007818BF044400F0E8F84E
:10162000401BA042FAD3B0BD0C0000207047000060
:1016300003490A68024208BF70470860FFF7F6BF17
:10164000140401402DE9FC4F624A05234FF0000BC2
:101650004FF0010A4FF0000890425F4A08BF032391
:101660000093002591460B6833FA05F208BFBDE8E8
:10167000FC8F0AFA05F213EA020E00F0A5804E680C
:1016800006F00304631E012B1AD80323D0F808C008
:10169000CF6803FA08F32CEA030C07FA08F747EAC5
:1016A0000C078760C6F3001707FA05FC476827EAAE
:1016B000020242EA0C026FEA030C42606A000AE08E
:1016C000032202FA08F2032C6FEA020C424602D10E
:1016D000424603241CE0C7688B6807EA0C07934066
:1016E0003B43022CC36013D16FF003060BF01C03C5
:1016F0000F2406EA55069C400644376A27EA04048C
:101700000F6907FA03F3234333624E6806F00304BC
:10171000036804FA02F203EA0C031A4316F4403F8A
:10172000026051D0EF4B1A6842F001021A601A6849
:101730004B46A9F57E7302F001020192019AAA08B4
:1017400053F822C0B0F1904F08D0BE4CA04207D051
:10175000234C009EA04208BF022602E0002600E0C3
:1017600001260BF00C070F24BC40BE404F462CEA6C
:101770000404344343F82240D9F800204C6842EA7C
:101780000E03E60358BF22EA0E03C9F80030A60391
:10179000D9F8042042EA0E0358BF22EA0E03C9F822
:1017A0000430E602D9F808200C4E42EA0E0358BF76
:1017B00022EA0E03C9F80830A402326842EA0E0396
:1017C00058BF22EA0E0333600BF1040B08F1020844
:1017D000013548E7000C0048000401400C040140BA
:1017E000000800481823002A08BF2823C15070476A
:1017F00099480068704700BF90F84120202A03D123
:1018000090F84020012A01D1022111E0242280F821
:1018100041200268136823F001031360136823F466
:101820008053136013681943734601F04EFC9E46C3
:101830000846704790F84120202A03D190F84020B4
:10184000012A01D1022110E0242280F841200268FF
:10185000136823F001031360136823F4706343EAF1
:101860000121734601F031FC9E4608467047000096
:1018700000B3B0B5044690F8410018B901F0D0FEAD
:1018800000F0B2F8242084F84100D4E90003D4E940
:101890000212056823F07063012A25F00105056036
:1018A0000361836823F40043836005D141F4004160
:1018B000816009E00120704741F40441022A8160FF
:1018C00004BF4FF40061416041680F4A04F1100504
:1018D00011434160C16821F40041C1602ECD114324
:1018E00041EA0321C160216A29430160016841F096
:1018F0000101016000202021606484F84110206310
:1019000084F84200B0BD00BF008000022DE9FE4F08
:1019100001F006FC0CD1DDF830B0BBF1000F09D0AE
:10192000DDF83480B8F1000F04D001F01FFD07D1BD
:10193000022502E001F0F8FD01252846BDE8FE8FF2
:1019400001F062FD01F0C6FD0028F6D1212001F072
:101950004BFE01F021F910B184F84050ECE701F0A2
:1019600086FD04D3FF20514601F0CFFD08E0608DD5
:1019700000214FF0007320850091C2B220465146ED
:1019800001F02EF90027FF26204641464A4601F085
:1019900087F90028D0D101F05FFC13D0000411D1E9
:1019A000204680210022434601F0BCFC0028C3D120
:1019B00001F05DFD02D301F0A0FD01E001F05FFD4B
:1019C00001F00EF9608D0028DED12046414601F07D
:1019D000E8FD0028B0D120682021024B01F0D4FCA2
:1019E000ABE700BF00E800FE10B586B00068134901
:1019F000884220D1124C206840F48020206020686A
:101A000000F4802000900420059003200490002022
:101A1000039012200290C0200190009801A909486B
:101A2000FFF710FEA06840F40010A060A06800F46A
:101A300000100090009806B010BD00BF0054004098
:101A400014100240000400481A48034900780A684C
:101A500010440860704700BFAC08002080B5CF4834
:101A6000016841F010010160032000F06FF80F20C1
:101A700000F004F800F020F8002080BD70B50D4E95
:101A800004464FF47A713078B1FBF0F0CB49096825
:101A9000B1FBF0F000F06EFC01250F2C08D838B92E
:101AA0004FF0FF3021460022002500F029F8746035
:101AB000284670BD0C00002082B00A48016841F041
:101AC00001010160016801F0010101910199416882
:101AD00041F080514160406800F0805000900098D3
:101AE00002B0704718100240002806D4734601F077
:101AF00010FB9E46014A42F82010704700E100E0CA
:101B0000F0B5184B4FF0FF361C68C4F30224E51EF5
:101B100084F0070438BF002506FA05F7BA43042C01
:101B200028BF042406FA04F4A14300F00F04A940DE
:101B3000043C11432344044A09010C33B0F1FF3F34
:101B4000C8BF83181970F0BD00E400E005494FF6E6
:101B5000FF030A681A4060F30A2203481043086032
:101B6000704700BF0CED00E00000FA052DE9FC41D4
:101B700004468078404EC00743D0306810F080584B
:101B800008D1306840F080503060306800F08050FC
:101B900001900198394F3868C00511D4386840F475
:101BA00080703860FFF724FE05463868C00507D40A
:101BB000FFF71EFE401B6428F7D90320BDE8FC8117
:101BC000706810F440700FD0616801F44071884271
:101BD0000AD02B49706801220A6000220A6020F4B2
:101BE0004071C007716038D16068716821F440713C
:101BF0000843B8F1000F706003D1306820F08050C6
:101C000030602068C10705D0A168726922F0030224
:101C100011437161810605D5E168726922F01002F5
:101C200011437161010605D52169326922F4F87208
:101C300011433161C10405D56169726922F4807272
:101C400011437161400405D5A069716921F4805187
:101C5000084370610020BDE8FC81FFF7C9FD05461F
:101C600041F2883770688007BED4FFF7C1FD411B81
:101C70000320B942F6D9EEE71C1002400070004084
:101C8000400442422DE9F84300285ED00D46434906
:101C90000446086800F00700A84209D2086820F04E
:101CA000070028430860086800F00700A8424CD1EC
:101CB0002068514B8946810705D5A1681A6822F032
:101CC000F00211431960C00736D1D9F8000000F0C6
:101CD0000700A8420CD9D9F8000020F007002843DB
:101CE000C9F80000D9F8000000F00700A8422CD184
:101CF0002068410705D5E1681A6822F4E0621143C3
:101D00001960000706D52069196821F4605141EA7D
:101D1000C00018601C4600F055F82168204AC1F345
:101D20000311515CC840254908601E480068FFF750
:101D3000A5FE0020BDE8F8836068022808D00128CD
:101D400026D153F8041C890306D40120BDE8F8838A
:101D500053F8041C8901F8D51968984621F003014D
:101D600008431860FFF744FD064641F28837606873
:101D7000D8F80010434601F00C01B1EB800FA4D05D
:101D8000FFF736FD801BB842F1D90320BDE8F88388
:101D900053F8041C8907D8D5DEE700BF00200240B5
:101DA000E05A00081000002004481349044A006863
:101DB0000968C1F30221515CC84070471C00002033
:101DC000F05A000810B50C490C480A6802F00C03E0
:101DD000082B08D10A4CC2F38343896AD203E35C1F
:101DE00002D40948584310BD064A01F00F01515C66
:101DF000B0FBF1F0584310BD0410024000127A000D
:101E0000646200087462000800093D002DE9FC418D
:101E100000287ED004460078AD4EC00744D07068DC
:101E200000F00C00042805D1306880033CD56068C0
:101E3000D0BB6EE001F068F902D17068C003F3D442
:101E400067682FB1B7F5A02F0AD0B7F5803F0BD048
:101E5000306820F480303060306820F4802006E064
:101E6000306840F480203060306840F4803030606A
:101E7000A068F16A21F00F010843F062FFF7B8FC97
:101E8000054677B1306880030ED4FFF7B1FC401BE4
:101E90006428F7D9F7E0FFF7ABFC411B0320642966
:101EA00035D830688003F6D42078800716D570685E
:101EB00010F00C0F05D001F027F961D17068C00354
:101EC0005ED43068800702D52069012821D160697D
:101ED000316821F0F80141EAC00030602078000745
:101EE0001AD4207840072AD4E7697FB101F00CF9B1
:101EF00073D1012F0DD0216A706800F480328A42BC
:101F000007D1616A00F47010884202D10020BDE858
:101F1000FC810120BDE8FC81A06900284CD06D48FF
:101F20000121C0F88014FFF763FC0546706A800742
:101F3000D7D4FFF75DFC401B0228F7D9A3E0F06976
:101F400010F0805808D1F06940F08050F061F069DD
:101F500000F08050019001985F4F3868C00521D48F
:101F6000386840F480703860FFF742FC05463868F6
:101F7000C00517D4FFF73CFC401B6428F7D982E06A
:101F800021695448002947D001210160FFF730FC46
:101F90000546306880079AD4FFF72AFC401B0228C8
:101FA000F7D970E0E068002846D0052856D001280F
:101FB00058D001F082F858E046480021C0F880145B
:101FC000FFF716FC0546706A80077FF58AAFFFF7BA
:101FD0000FFC401B0228F6D955E03E4900208846F8
:101FE0000866FFF705FC0546022F0AD14746306810
:101FF000800154D5FFF7FCFB411B03200229F6D9D1
:1020000085E7306880017FF581AFFFF7F1FB411B69
:1020100003200229F5D97AE700210160FFF7E8FBE8
:102020000546306880077FF559AFFFF7E1FB411B9C
:1020300003200229F5D96AE701F03FF83062FFF783
:10204000D7FB054641F28837306A80071ED5FFF777
:10205000CFFB411B0320B942F6D958E7306A40F064
:1020600004003062306A40F001003062FFF7C0FBCC
:10207000054641F28837306A800707D4FFF7B8FB7E
:10208000401BB842F7D90320BDE8FC81B8F1000F2E
:102090007FF42AAFF06920F08050F06124E7D4E9A2
:1020A0000801726822F47412114308437060012021
:1020B0003866FFF79DFB0446306880013FF526AF88
:1020C000FFF796FB011B03200229F5D91FE700BF8C
:1020D00000100240000042420070004040B1F8B5DC
:1020E0000446406A30B10020206104F1140007E08A
:1020F000012070476068B0F5827F03D004F11C00B6
:10210000002101600025A56294F85D0020B92046F9
:1021100084F85C5000F04CF8022084F85D002068E0
:10212000E1680268B1F5E06F41F4006301F47061A9
:1021300022F04002026098BF01252A03B3F5706FB8
:102140001CBF0023A362D4E90135D4E9046711431D
:1021500003F4827305F404452B4406F002052B4476
:1021600007F001052B44A56905F400763344E669C0
:1021700006F038063344266A06F080063344A66A21
:1021800006F40056334303600423626A03EA1543EE
:10219000194302F010021143626B02F0080211436E
:1021A000416000200121206684F85D10F8BD000028
:1021B000FEB500681249884220D11248416841F4B6
:1021C00080514160416801F4805101910199016899
:1021D00041F480210160006800F480200090052017
:1021E00005900320049000200390022002903820E4
:1021F0000190009801A90448FFF724FA06B080BDB9
:102200000030014014100240000400482DE9F8435A
:1022100001F049F804BF0220BDE8F8834FF001093E
:102220001D4616460F4684F85C90FFF7E1FA80469B
:1022300094F85D00012843D1002F43D0002E41D0F7
:10224000032084F85D0000202066E687A687A76348
:10225000A4F844002064C4E91300A4F84600A1686F
:102260002068B1F5004F05D101F074F9016841F41F
:10227000804101600168490601D400F0CDFFE168AA
:102280006268B1F5E06F1FD90AB1012E01D101F0EA
:102290000FF86E1CE08F002851D0206881688907F4
:1022A00008D4FFF7A5FA002EF4D0A0EB0800A8424E
:1022B000F0D35BE000F078FFE08F0138E087E9E7DA
:1022C000022054E0012052E04FF6FE710AB1012EC7
:1022D00011D1E28F022A05D337F8022BC2604FF6E4
:1022E000FE7004E03A780273481CA26B571CA76387
:1022F000E28F1044E0876E1C4F1CE08FF8B120681D
:102300008168890708D4FFF773FA002EF5D0A0EB97
:102310000800A842F1D329E0E18F022904D300F09C
:1023200043FF4FF6FE7006E0A16B09780173A06BC6
:102330000130A0633846E18F0844E087DDE720469E
:102340002946424601F072F908B120202066A068B3
:1023500038B9002000902068C16800918068009022
:102360000098206E002818BF012000E0032000F034
:1023700046BF0000411E0020B0EB116F1CBF0120C2
:102380007047044AF023516003490B7007219060A5
:102390001160704710E000E023ED00E070477047E7
:1023A0007047000070B590F83C20012A01D102214D
:1023B00031E091E83C00194E25F47C5524F470542A
:1023C00033402C4322F4772223435E4C1A430B699B
:1023D00023F476231A434B691A438B6A22F474223E
:1023E00023F470231A438B6942EA03430268A24232
:1023F0000DD1D1E90745496A094E23F07C7306EAFD
:102400000151194324F00073194341EA05030021E7
:1024100080F83C105364084670BD00BFFF87F0FF92
:102420000000F0FC70B590F83C300222012B26D061
:1024300080F83D20434C026855689368A24203D15E
:102440004E6825F4700535430E6825F07005354358
:10245000B2F1804F556007D0384DAA4204D0384DB4
:10246000AA4201D0A24204D1896823F08003194313
:1024700091600022012180F83C2080F83D10104638
:1024800070BD00BF58B110B501F00FF803D100F0D6
:1024900076FF00F007F801F0BCF800F046BE01201E
:1024A00070470000E0B50068BF49884216D0B0F11F
:1024B000804F17D10C480022416841F00101416072
:1024C0000021406800F00100019001981C20FFF7F6
:1024D00017FB1C20BDE88C40FFF706BB024800F04C
:1024E000D6FD00988CBD00BF1810024090F83D103A
:1024F00001291CBF01207047022180F83D100168AE
:10250000C868B1F1804F40F00100C86008D00B48A6
:10251000814205D00A48814202D00A4881420AD14C
:102520008868094A734600F099FF9E4602D0B2F5CA
:10253000803F00D1704700F0DABF00BF00040040C8
:1025400000400140002C014007000100016841F2F9
:102550001113CA6822F00102CA600A6A1A4208D13D
:102560000A6A40F244431A4203D10A6822F0010287
:102570000A6001F001B8000010B500F089FF51D0E9
:1025800084F83D000120294B84F83C0020688268D3
:102590001A4082600A68C2B1102A16D0202A14D0CC
:1025A000302A12D0402A17D0502A1ED0602A25D0B7
:1025B000B2F5005F2ED0B2F5805F30D0702A32D1F4
:1025C00000F0B4FE41F0770128E0816821F070014D
:1025D000114341F0070121E000F0AAFF2068816863
:1025E00041F0470121F0300118E000F0A1FF206820
:1025F000816841F0570121F020010FE04B68CA6863
:10260000194601F012FC2068816841F0670121F051
:10261000100103E000F08AFE41F480418160002057
:1026200000F0A3FF10BD0120FAE700BF8800FEFF05
:10263000704710B5044600680169890712D5C16862
:1026400089070FD56FF002010161012121778069AF
:10265000800702D000F065FF01E000F0AAFE002034
:10266000207720680169490713D5C168490710D54B
:102670006FF00401016102212177806910F4407F2D
:1026800002D000F04EFF01E000F093FE0020207722
:1026900020680169090712D5C16809070FD56FF0D5
:1026A0000801016104212177C069800702D000F090
:1026B00038FF01E000F07DFE0020207720680169EE
:1026C000C90613D5C168C90610D56FF010010161A4
:1026D00008212177C06910F4407F02D000F021FF6B
:1026E00001E000F066FE0020207720680169C9073C
:1026F00009D0C168C90706D06FF001010161204609
:1027000000F064F920680169090609D5C168090665
:1027100006D56FF0800101612046FFF740FE20687A
:102720000169C90509D5C168090606D56FF480712C
:1027300001612046FFF732FE20680169490609D58C
:10274000C168490606D56FF040010161204600F0DE
:102750003EF920680169890602D5C168890600D45E
:1027600010BD6FF0200101612046BDE81040FFF769
:1027700017BE0000FEB500680B49884211D1B84869
:1027800000F085FC012005900020CDE90300022027
:1027900002904FF400700190009801A90348FEF7E1
:1027A00051FF06B080BD00BF004801400004004852
:1027B00070470000B0B500F0F7FE04BF0220B0BDC6
:1027C0000D4601204FEAB201052984F83C0048D8A3
:1027D000DFE801F0030B131B23332068294601F0C7
:1027E000F9F9206850F8181F1EE02068294601F00A
:1027F0002BFA206850F8181F26E02068294601F0BF
:1028000055FA206850F81C1F0EE02068294601F098
:1028100087FA206850F81C1F16E02068294601F04E
:10282000ABFA206850F8541F41F0080101600168BC
:1028300021F00401016029690FE02068294601F0B8
:10284000BDFA206850F8541F41F40061016001682E
:1028500021F4806101602969090202681143016065
:102860000020002184F83C10B0BD58B110B500F034
:102870001CFE03D100F083FD00F006F800F0C9FE55
:1028800000F053BC0120704770477047B0B5044654
:1028900051B1081F00F094FC16D8DFE800F0020CDC
:1028A0000F1204F13F0211E094F83E00012819D103
:1028B00000F033FE23E004F1400207E004F141029E
:1028C00004E004F1420201E004F143021278012A1B
:1028D00008D1032808D8DFE800F0020A0D1000F044
:1028E00064FD0CE00120B0BD00F082FD07E000F0C7
:1028F00093FD04E000F080FD01E000F081FD00F0B8
:102900004BFE2168304800F008FD06D800F0AAFD13
:102910001EBF486C40F400404864B1F1804F08D0BD
:102920000948814205D00948814202D008488142C5
:1029300007D18868074A00F091FD04D0B2F5803FC6
:1029400001D000F00DFCB0BD00040040004001408B
:10295000002C014007000100B0B500F070FC2068B9
:10296000194900F018FC0AD800F0F9FD07D000F072
:1029700070FD04D100F088FC01D100F052FC00F0A1
:1029800068FD04D100F080FC01D100F0F3FC4FEAB7
:10299000B500042807D8DFE800F003090C0F120087
:1029A00000F069FD0DE000F017FD0AE000F09CFC6E
:1029B00007E000F0ABFC04E000F087FC01E000F071
:1029C000E7FD0020B0BD00BF00D4FEBF70477047D8
:1029D00010B540B10446806F08B900F0FFFD00F06B
:1029E00058FC012801D1012010BD606A08B100F037
:1029F00091FC00F07DFC21F02A01816000F0B6FB23
:102A0000BDE8104001F076BAFEB50068134988426F
:102A100021D1DD48816841F400318160816801F491
:102A2000003101910199016841F4003101600068B1
:102A300000F400300090072005900320049000204F
:102A40000390022002900C200190009801A94FF001
:102A50009040FEF7F7FD06B080BD00BF0044004087
:102A6000141002402DE9F8430446806F202807D156
:102A70000E4641B1174632B194F87400012805D1D1
:102A80000220BDE8F8830120BDE8F8834FF000097B
:102A900001201D46C4F8809084F874002120A067AE
:102AA000FEF7A6FEA4F852708046A4F85070A06805
:102AB000B0F5805F01D1206908B1002701E03746F9
:102AC000002684F87490B4F85200B8B120468021F2
:102AD00000F0F6FBB8B926B116F8010B216808859D
:102AE00006E037F8021B206800266FF35F2101859E
:102AF000B4F852000138A4F85200E4E7204640211F
:102B000000F0DEFB10B10320BDE8F8832020A067B1
:102B10000020BDE8F883FEE700688169890744BFAB
:102B2000002181628169C90703D1816941F00101F6
:102B300081617047F8B5044600680E468169C90690
:102B40005CBF0020F8BD41681546890101D400F042
:102B500030FD771C816989060AD4002FFAD0FEF770
:102B600047FE411B2020B1420ED86EB12068F1E72C
:102B70001021C1612021C16100F052FC2068054A8A
:102B80004168114041600420616C084300F021FB62
:102B90000120F8BD00E800FE2DE9FC4104460F4885
:102BA00015461E46DAB24FF0807300F0F0FA00F0DE
:102BB00075FC10B10120BDE8FC81012E03D000F0AE
:102BC0000FFC0028F6D100F0DCFC8021009700F01B
:102BD0001BF8002818BF0120BDE8FC810020008000
:102BE00010B5029C00686FF39F2141EA02414268E0
:102BF00023431943034B22EA54521A4011434160C4
:102C000010BD00BF009C00FC2DE9F843DDF82080DA
:102C10001D4616460F4681465C1CD9F800008069A7
:102C20003840C01BB0FA80F04009B0421AD1002CE5
:102C3000F3D0FEF7DDFDA0EB0800A84201D8002D7F
:102C4000EBD1D9F8440040F02000C9F8440020201E
:102C500089F84100002089F8400089F842000120ED
:102C6000BDE8F8830020BDE8F88370B515460E4630
:102C7000044620688069800644BF002070BD00F0D3
:102C8000D2FB58B9FEF7B4FD401BB04201D8002E6C
:102C9000EFD1606C40F0200000F09BFA012070BD85
:102CA000F8B515460E4604464F1C2068806980071B
:102CB00044BF0020F8BD00F0B6FB68B9002FF4D087
:102CC000FEF796FD401BB04201D8002EEDD1606C9E
:102CD00040F0200000F07DFA0120F8BD10B58AB068
:102CE000002418210994CDE9074401A8FDF79FFAB3
:102CF000194801224FF0A041C0E90A24C261042210
:102D000080F8204080F8304044630483C0E9001418
:102D1000C0E90244C0E90442FEF71CFA08B1FDF71D
:102D20000AFF0D48079407A9FDF70EFF08B1FDF74C
:102D300002FF00200121029106210390CDE9040049
:102D400006900548019101A9FDF76AFF08B1FDF75A
:102D5000F2FE0AB010BD00BF4C060020E0B54B48A3
:102D60000022016841F0010101600021006800F0CB
:102D70000100019001980B20FEF7C2FE0B20BDE878
:102D80008C40FEF7B1BE00BF141002402DE9F04F99
:102D900087B000263D483E4C0022CDE9056601681B
:102DA00041F400210160016801F4002101910199C1
:102DB000016841F400310160016801F400310191C2
:102DC0000199016841F480210160016801F48021CA
:102DD00001910199016841F48011016048F20201FA
:102DE000006800F48010019001984FF09040A047D7
:102DF000284F4FF4AE51002207F580652846A047C2
:102E000007F5006B04210022BA465846A0474FF44C
:102E100088194FF0010804961F4C4FF09040CDF8F0
:102E20000C90CDF8088002AF3946A04748F2020066
:102E300000F027F94FF09040A04706203946CDE931
:102E4000039602905046A0474FF4AE5000F019F997
:102E50002846A047042000F014F95846A0470F4C1C
:102E6000062000210022A0470D4D0620A84707207C
:102E700000210022A0470720A847082000210022A7
:102E8000A0470820A84707B0BDE8F08F1410024003
:102E9000E51700080004004845160008011B00085B
:102EA000E91A000810B5124C01200021114A124BFA
:102EB000C4E9021004F110001421C4E90032FDF746
:102EC000B6F92046FEF7D4FC08B1FDF734FE0848F9
:102ED0000021FEF791FC08B1FDF72DFE044800210A
:102EE000FEF7A8FC18B1BDE81040FDF724BE10BDE8
:102EF000E00600200E09002000540040B0B5104844
:102F000000214FF400724FF4E0630E4D4FF48274D1
:102F1000C0E90213C0E9062108220723C0E90054D2
:102F2000C0E90411C0E90811C0E90A13C0E90C1294
:102F3000FFF7D4F818B1BDE8B040FDF7FCBDB0BD57
:102F40002C07002000300140B0B592B068462C211B
:102F5000FDF76DF91D481E4B00216322C0E90031C9
:102F6000C0E90212C0E904118161FFF78BFA08B1D0
:102F7000FDF7E1FD1548FFF778FC08B1FDF7DBFD33
:102F8000602018210B900BAC201DFDF750F90F4865
:102F9000214600220025FFF70DFC08B1FDF7CBFD0F
:102FA0006C4614212046FDF742F94FF400502146AB
:102FB0000A95069505900548FFF7F4F908B1FDF765
:102FC000BAFD0248FFF7D6FB12B0B0BD9007002053
:102FD0000048014010B588B01548002140F2E732A2
:102FE00007234FF080440791CDE9051102918161DB
:102FF000C0E90043C0E902120161FFF743FA08B1DA
:10300000FDF799FD4FF480500490094804A9FFF79B
:10301000B3FA08B1FDF78FFD00200390019004483A
:1030200001A9FFF7FFF908B1FDF785FD08B010BD54
:10303000DC07002010B50C480C4C00210C224FF48A
:103040001643C0E90043C0E90211C0E90412C0E917
:103050000611C0E90811FFF7BBFC18B1BDE810402C
:10306000FDF769BD10BD00BF2808002000440040E6
:10307000FEE7FEE782B2284621464FF47A73FFF757
:10308000F1BC39460596CDE9038602907047016888
:1030900041F480210160006800F4802000907047B6
:1030A00007EB8000B8EEC00A90ED001A20EE080A87
:1030B00020EE010A80EE090A7047306A20F0010014
:1030C0003062306A20F0040070471160116841F0EE
:1030D000010111600021202280F8401080F8412079
:1030E0007047206850E8020F216820F0010041E895
:1030F0000202002A70472046FDF7A4B800250168A7
:103100004A630021FFF7C2BB706800F00C0008287A
:10311000704700F01F010122400902FA01F17047D7
:10312000044690F8410020287047012084F84800A8
:1031300084F83E0084F83F0084F8400084F84100A1
:1031400084F8420084F8430084F8440084F8450081
:1031500084F8460084F8470084F83D00002010BD44
:10316000086840F00100086000207047016841F0E5
:103170000101016020467047216C41F480412164C7
:10318000616C41F0080161644FF480617047009008
:103190002046FFF725BD01444FEAB12107297047BA
:1031A00094F83C0001287047A16B31F8022BC260F3
:1031B000A1637047016C41F0200101640121704757
:1031C0004FEAB00003287047816801F0030101292C
:1031D00070476064202084F84100002084F840009B
:1031E00084F842007047816841F0040181607047B3
:1031F00020464FF4C06132462B4600F02DBA002124
:1032000084F85C1084F85D90BDE8F88300222B46BA
:103210000090204600F026BF016841F040010160A7
:103220007047416C21F4004141647047016821F40A
:1032300000510160016841F400510160704704468B
:10324000006800220D4600F0B5BCC36802F40052CD
:1032500003F44063D2187047616A206811F8012BAB
:103260008262608D013860856162208D0138208521
:10327000618D002970472D9938602A9878602998C7
:10328000B8602898F8607047016A40F244421142E1
:1032900070472420A0672068016821F001010160C7
:1032A000204600F04FBE044690F85C0001287047AD
:1032B00037F8021BC160A763E08F0138E0877047D1
:1032C00000224346009500F0CDBE012084F8410065
:1032D0007047206C40F6017188437047206E40F0C3
:1032E00020002066032070BD012084F83F00704755
:1032F0002068416821F49041416081687047206CEA
:1033000004F1440140F0100020647047012084F86B
:1033100040007047204600F099BD08444FEAB020B5
:1033200007287047CDF80090FFF76EBCD1E9012364
:10333000C9681A4342EA0121826822F47F4211439C
:103340008160816870470446006880684007704764
:103350004268B1F5827F22F0E002426070474FF090
:1033600090404FF400410122FEF73CBA94F840002F
:1033700001287047016821F00101016070470020B9
:1033800084F83C00204670470025C16142681A401D
:10339000426084F8411084F8405084F842507047ED
:1033A000204631462A4600F0B1B9022084F83F0099
:1033B00070474DF808ED2046FFF7FAF920465DF812
:1033C00008EBFFF762BA82B2284621464FF47A73BF
:1033D00030472046FDF78DBA012084F8430070473E
:1033E0002068290A3A46816220464146FFF758BCC8
:1033F000022084F843007047022084F8410070479F
:10340000022084F84200704701251F4616468A466E
:1034100084F84050FEF7ECB9022084F84000704771
:103420002046FFF779BB204631462A46FFF782BB8C
:10343000D0F820C046680C688B68456D02444FEA9E
:10344000B227072F704782B2284621464FF47A737D
:103450003847016A41F211121142704702400020C0
:10346000062A704705FA00F010F0E10F7047608DF2
:10347000B0F5807F7047012084F83E007047608D72
:1034800051464FF000732085C2B220460097704726
:1034900090F83C2004460220012A7047DDE90887A5
:1034A000204641463A46FFF7FBBB044690F83D00F4
:1034B0000028704702460B462046514601F072BA7A
:1034C000D1F800C01F2604EB43040CFA04F506FAF9
:1034D00004F470478146009020464FF400410122D9
:1034E0001923FFF791BB41E80002002A70470868E2
:1034F00040F00100086000207047268500972046B4
:103500005146FF224FF080737047FF224FF08073C7
:1035100020850020009020467047022084F83E005D
:1035200070472046FFF784B84FF40070606470471E
:103530004B68CA68194600F067BCB04202620A686C
:103540008B68046A4568704703224FF47A732046FB
:10355000FEF75CBE016821F0400101607047012266
:1035600002FA01F111F0E10F7047002184F83C10DC
:10357000012184F83D107047012180F83D100020A2
:1035800070472068E9B200224346816220467047B6
:10359000012084F84200704720680122012500F0D4
:1035A00009BB4A46FFF761BB044690F83C0001287E
:1035B0007047416841F4804141607047ADF80400B4
:1035C0004FF09040FEF70EB9206C40F010002064E0
:1035D000606C40F0010060640120B0BD002084F800
:1035E00074002046FFF710BA0E99002532463B467C
:1035F00084F84100402084F842006564C4F824B097
:103600006563A4F82A808846CDE900192046514612
:1036100070470220211D84F83D00206800F08ABA1E
:10362000002084F8400020467047704770B515466A
:103630000E464FF4C051044632462B4600F00CF8BB
:1036400028B9FFF7ADFE10B9FFF7D2FD08B1FFF7BB
:1036500045BE002070BD00002DE9FE4380460020DD
:103660001E4617460D468DF80700FEF7C1F8301AC2
:10367000C419FEF7BDF8814646482321013700688A
:103680004843000D60430290D8F8006030468168DE
:10369000294219D0B5F5C06F04D1317B8DF80710E0
:1036A0009DF80710002FF2D0FEF7A2F8A0EB09005A
:1036B000A0420CD20298029901390291002808BF59
:1036C0000446D8F80000E2E70020BDE8FE83D8E910
:1036D0000001FFF73DFE09D1D8F80810B1F5004F01
:1036E00002D0B1F5806F01D1FFF734FFD8F8281070
:1036F000B1F5005F01D1FFF799FD002088F85C006B
:10370000012088F85D000320BDE8FE83F8B515466A
:103710000E460446FEF76CF8281A8719FEF768F87B
:1037200005461C4801360068C0F3CB307843009052
:103730002068816809065CBF0020F8BD002EF8D023
:10374000FEF756F8401BB84207D20098009901399D
:103750000091002808BF0746EAE7D4E90001FFF717
:10376000F7FD08D1A168B1F5004F02D0B1F5806F27
:1037700001D1FFF7EFFEA16AB1F5005F01D1FFF7BC
:1037800055FD002084F85C00012084F85D000320D2
:10379000F8BD00BF1C00002070470000022888BF51
:1037A0007047F8B50F49D54C0F4F01EAC0064FF4EA
:1037B00080700421F040C5B204F580602A46B84705
:1037C0004FF480304FF48051F040C2B22046B847E9
:1037D00020464FF480612A463B4601B0BDE8F040E8
:1037E000184700BFF8FFFF00E5170008FEF72CB9E7
:1037F000B0B596B00CAC1821201DFCF718FD68463A
:1038000018210430FCF713FD4FF40020102100258F
:103810001590022011910121149513900C902046CF
:103820001091FEF7F3FA18B1EFF3108072B6FEE7CD
:103830000F200895CDE909550B950021079007A8A1
:10384000FEF720FA18B1EFF3108072B6FEE74FF4DE
:1038500080700490A0200090002003906846FEF73E
:1038600085F918B1EFF3108072B6FEE716B0B0BD5F
:103870000248016841F470010160704788ED00E082
:103880002DE9F0412DED048B954C2088042805D1BD
:10389000994D2869C0B100206861ECE0914D28681D
:1038A000C82800F0C080012800F0CB80002840F03C
:1038B000D78028688E490122012601EB40018D48FE
:1038C000FDF77EFD2680D3E06868092800F3DA80E2
:1038D0008A4C402100222046FDF784FFDFF8208239
:1038E000296A804E884F9FED878A9FED889AD8F885
:1038F00000006962C8F80400686896ED000AFFF7E6
:10390000CFFB01F0CDF988ED000A96ED000A68685A
:10391000FFF7C6FB01F0BAFA85ED080A2046402100
:10392000012298ED008AFDF75DFF9FED790A28EEF0
:10393000000A01F05DFA10EE100AFCF7BFFD9FEDE2
:10394000660B53EC102BFCF784FCFCF798FD6649E2
:103950009FED701A09684863686896ED002A07EBC6
:103960008000B8EEC22A90ED000A81EE001AB4EE93
:10397000421AF1EE10FA80F2928095ED061A9FED50
:10398000672AB1EE083A21EE021A20EE011A81EE02
:10399000031A85ED0A1A95ED071A21EE021A20EE98
:1039A000010A80EE030A85ED0B0A95ED0A0A95EDF2
:1039B0000A2A95ED0B1A95ED0B3A21EE031A00EE4B
:1039C000021AB1EEC10AB4EE400AF1EE10FA7CD64A
:1039D0009FED531A6868534980EE010A01EB80009D
:1039E00080ED000A95ED0B0AD5ED0A0A01F002F808
:1039F0009FED4E1A68684C494FF07E5220EE010A46
:103A00009FED4B1A01EB8001013080EE010A81ED40
:103A1000000A002131606961C8F800202962A961AB
:103A20006860E9614DE0304800210026FEF794FF10
:103A30000020FFF7B3FE2D48FEF788FD03202E601F
:103A40000CE0294864210122006841632849286864
:103A500001EB40012748FDF7B3FC0220208007E07E
:103A600028682349022201EB40012248FDF7A8FC07
:103A70002868013028601D48BDEC048BBDE8F0418A
:103A8000FEF7D7BD18480021FEF766FF1748FEF77E
:103A90005DFD0020FFF782FE05202080EBE79FED13
:103AA0001E1A81EE000A96ED001AB8EEC11AB4EEA5
:103AB000410AF1EE10FA04DA0E480D490222FDF730
:103AC0007FFC306801303060D5E7B0EE410A01F08C
:103AD000A5FA7DE700BF00BF0000000000004E40D7
:103AE000200000202400002090070020DC07002098
:103AF000BC0400204C0600207C0000200008004888
:103B000004000020C70EC9408462000800007A4407
:103B10000000204200401C4600007A456F12833AA4
:103B2000000070425000002028000020000034C334
:103B3000560E494070B5754A0368904217D01C4C28
:103B400040F48065A54203D14D6823F070032B43F8
:103B5000B0F1804F0FD0A0420DD06D4CA0420AD0E2
:103B60006C4CA04207D06C4CA04204D007E04C68DB
:103B700023F070032343CC6823F4407323434E693E
:103B800023F080030C688D68334390420360C56264
:103B9000846208D05E4A904205D05E4A904202D0CC
:103BA0005D4A904201D1096901630121416170BD03
:103BB0000004004010B501F01F010123046A8B408E
:103BC00002FA01F124EA03030362026A114301626B
:103BD00010BD0000F0B5026A4C4E22F001020262F4
:103BE0000A688B68046A456824F0020423438469E8
:103BF000B04208D0464FB84205D0464FB84202D036
:103C0000454FB84207D1CF6823F00C0327F00407D3
:103C10003B43B04208D03E4EB04205D03D4EB0428C
:103C200002D03D4EB04205D1D1E9056725F440757B
:103C300035433D434560394D2C40224382614968FC
:103C400041630362F0BD00BFF0B5026A2F4E22F05F
:103C50001002FFF772FC24F0200444EA0313846985
:103C600009D02B4EB0420ED02A4EB0420BD02A4E75
:103C7000B04208D00FE0CE686FF0400723F0C003D9
:103C800007EA06163343D1E9056725F4406545EA9E
:103C9000860545EA87054560364D2C4044EA0222F8
:103CA0008261496881630362F0BD00BFF0B5026ABA
:103CB000164E22F48072FFF740FC24F4007444EAAC
:103CC0000323C46909D0124EB0420ED0114EB04247
:103CD0000BD0114EB04208D00FE0CE6840F2FF4743
:103CE00023F440633602BE433343D1E9056725F42C
:103CF000405545EA061545EA07154560074D2C4035
:103D00002243C2614968C1630362F0BD002C0140D7
:103D10000040014000480140004401408CFFFEFF8C
:103D2000F0B5026A22F480520262354AD0F820C00F
:103D300046680C688B68C56902444FEAB227072FB2
:103D400009D80122BA4012F0E10F1EBF4A6926F4D9
:103D5000804646EA8216074A46602A4042EA042222
:103D6000C261496801642CF4005141EA03310162E7
:103D7000F0BD00BFFF8CFFFEF0B5026A22F4803276
:103D800002621F4AFFF754FB09D80122BA4012F021
:103D9000E10F1EBF4A6926F4803646EA0226064A2B
:103DA00046602A4022434265496881652CF400310F
:103DB00041EA03410162F0BD8FFFFEFFF0B5026AE8
:103DC00022F4801202620E4AFFF732FB09D8012268
:103DD000BA4012F0E10F1EBF4A6926F4802646EA77
:103DE0008226084A46602A4042EA0422426549681F
:103DF000C1652CF4001141EA03510162F0BD00BF1E
:103E000000D4FEBFFF8FFFFE10B5036A046A24F0E2
:103E100001040462846924F0F00444EA021282611D
:103E200023F00A021143016210BD036A23F010035C
:103E30000362836923F4704343EA0232036A8261B6
:103E400023F0A00242EA01110162704710B5416AF5
:103E5000CA0706D00268836A546824F400342343F6
:103E600053608A0706D50268C36A546824F4803414
:103E7000234353604A0706D50268036B546824F451
:103E80008024234353600A0706D50268436B5468B5
:103E900024F4004423435360CA0606D50268836BAA
:103EA000946824F48054234393608A0606D50268FC
:103EB000C36B946824F40054234393604A060FD5DF
:103EC0000268036C546824F480141C43B3F5801F0B
:103ED000546005D1436C546824F4C00423435360F8
:103EE000090606D50168806C4A6822F40022104356
:103EF000486010BDBCB504460020C4F88000FDF742
:103F000077FC054620680168090707D56FF07E40F9
:103F10004FF40011FFF77AF950B9206800684007A4
:103F200008D56FF07E404FF48001FFF76FF908B1BC
:103F30000320BCBD2020A067E067002084F8740047
:103F40002066BCBD70B5044600683C4E04F1080311
:103F50000ECB056835406669194341EA0603E169FD
:103F60000B432B430360436823F440531A434260DE
:103F7000A269236A1A43836823F430631A43304BDF
:103F80008260002298420ED02E4B98420BD02E4ACF
:103F9000904207D12D482EA2006800F0030052F88D
:103FA000202000E010222E48B1F5004F0CD1012155
:103FB000082A3DD8DFE802F0053C1B3C153C3C3CA0
:103FC0001900FDF7F1FE0EE00121082A30D8DFE8E4
:103FD00002F0052F222F1C2F2F2F2000FDF7E4FECB
:103FE00015E0FDF7EFFE10B91FE04FF400406168E7
:103FF0004A0802EB4000B0FBF1F04FF6F0710140CF
:1040000015D0C0F3420008430DE0FDF7DBFE10B908
:104010000BE04FF40040616800EB5100B0FBF1F0A1
:1040200080B2102803D32168C860002100E001217C
:104030000020C4E91900084670BD00BFF369FFEF16
:104040000044004000480040003801403010024069
:104050000000000004000000080000000200000052
:1040600000127A002DE9F843DDF82090044600683C
:10407000984616460F4609F10105C1693940C91B2A
:10408000B1FA81F14909B1421ED1002DF5D0FDF7F9
:10409000AFFBA0EB0800484519D8B9F1000F16D0C6
:1040A000206801684907E8D5C1690905E5D54FF4DD
:1040B0000061016250E8000F216820F4D070FFF722
:1040C00012FA15D02068F5E70020BDE8F8832068D3
:1040D00050E8000F216820F4D070FFF704FAF6D101
:1040E000FEF7FFFFFCD12020A06704F17C0007E071
:1040F000FEF7F7FFFCD12020A067E06704F1800005
:10410000002184F87410202101600320BDE8F883A9
:10411000FEE7000000000000DCB0FDF79FFCFFF7A9
:1041200067FBFEF733FEFEF7E9FEFEF70DFFFEF735
:10413000B9FEFEF713FEFEF7D1FDFEF74BFFFEF7CB
:1041400079FF00F04DFBE94CDFF8D8544021012203
:104150002046A847204680210122A84720464FF448
:1041600080710122A8470220FCF714FCDFF8B80494
:104170009FEDDF0B2F900FF2B040D0E90112CDE997
:1041800030128189807B8DF8CA00DFF8AC04ADF86D
:10419000C810D0E90041D0E90223008ACDE92A14F1
:1041A000CDE93441D4492790ADF8E000DFF8900420
:1041B000CDE92832CDE936233E917921ADF8FC10C6
:1041C00090E81E00008ACDE92343CDE9252139ADD1
:1041D0002290ADF8F4001EC543AC53EC102B0FF247
:1041E0006441204600F0DEFBFEF785FFDFF87854DF
:1041F00082B221464FF47A732846FEF733FC2FA98A
:10420000DFF86884DFF82495DFF824B59FEDBC8BD8
:10421000DFF8ACA401F13C0001F114072D9001F18D
:1042200028002C972E90DFF8FC0401681F9141684C
:104230001E9181681D918189807B1B90DFF8E804C5
:104240001C9101681A91416880681890DFF8CC04CD
:10425000199101681791416816918168007B14904B
:10426000DFF8940415910168139141681291018956
:10427000807A1090DFF85C04119101680F91416819
:104280000E918168007B0C90DFF84C040D91016861
:104290000B914168806809900FF240400A91416893
:1042A00008918168808906900FF2C43007914168B7
:1042B000008905910490B8F800000138042800F244
:1042C0008A81DFE800F0031C3996D7000020A8F8A7
:1042D00000001F9838601E9878601D98B8601C9880
:1042E000B8811B98B8732020ADF8F800ADF8E40051
:1042F0001A982F9019983090189831906BE14FF0E0
:10430000000BDFF81C14A8F800B017982F9016982F
:1043100030901598319014988DF8C800D8F8042082
:104320002E9800F03FFB8DF8F8B08DF8E4B0DFF880
:1043300000B4DFF8F893F0E000203A22A8F800007B
:104340002B98FEF798FF13982F90129830901198A1
:10435000ADF8C40010988DF8C60027983882B74889
:1043600008607920888026982E99086025984860F2
:10437000249888602398C86022980882DF492046E4
:10438000FBF72EFFDE4E2046B047DE4EFFF71BF850
:10439000DD4920462D223746FBF722FFD84E204626
:1043A000B047FFF750F8D94920462622FBF718FFFF
:1043B0002046B047D34FFFF746F8D548D549028885
:1043C000204600F0EFFA2046B047CE4EFEF7FBFF46
:1043D0000126C82E00F09880CD48CF4930F816202D
:1043E000204600F0DFFAFEF786FEFEF743FE0136B8
:1043F000EFE70F98B94938600E9878600D98B8606B
:104400000C9838730B982F900A9830900998319037
:104410002E98016008994160079981600699818111
:10442000B2480068002800F0D0806FF0030101EB73
:1044300080069B488059FCF741F8CDE9201046449E
:10444000306BFCF73BF80746B0688B46FCF736F854
:1044500041EC100B4BEC117B2D98A549DDE9203286
:10446000DFF8CCB2DFF8C4922C9F8DED001B8DEDF0
:10447000020BAEE00020A8F800002B982E9AFEF761
:10448000FAFE279838827A482F9005983090049841
:10449000ADF8C4002698106025985060249890606C
:1044A0002398D0606548086079208880229873A19D
:1044B000108253EC182B204600F074FAFEF71BFE16
:1044C000FEF7D8FD0426282E29D075488059FBF721
:1044D000F5FF02460B46204672A100F063FAFEF794
:1044E0000AFEFEF7C7FD0436EDE700BF00080048EE
:1044F0003333333333332B40456E6A6F00BF00BF15
:10450000000000000000F03F0A20ADF810016748ED
:104510004390FEF7F0FDFEF7ADFD2C9F5BE0634896
:1045200000268DF810614390FEF7E5FDFEF7A2FD31
:10453000D8F83000FBF7C2FF02460B4620465CA1CC
:1045400000F030FAFEF7D7FDFEF794FD242E0CD0D4
:1045500008EB0600406BFBF7B1FFFEF7ABFFFEF781
:10456000CAFDFEF787FD0436F0E700208DF8100144
:104570004E484390FEF7BFFDFEF77CFDD8F80800DB
:10458000FBF79CFF02460B4620464EA100F00AFABC
:10459000FEF7B1FDFEF76EFD0C26302E0BD058F85D
:1045A0000600FBF78BFFFEF785FFFEF7A4FDFEF785
:1045B00061FD0436F1E70A20ADF810013B48439055
:1045C000FEF799FDFEF756FD05E02D98494953EC9D
:1045D000182B00F0E7F9002000F0F4F80520052181
:1045E000C847DBE90012534E2FA80123B04705202E
:1045F0001421C847DBE9001238460123B0470520E3
:104600002321C847DBE900122E980123B04705207B
:104610003221C847DBE900122D980123B04700F092
:1046200029F948E6E517000857656C636F6D65204A
:104630002D20474549490000D4630008456E6A6F44
:10464000E863000857656C636F6D65202D20474552
:1046500049490A4964656E746966204D43432025C3
:10466000322E32660A0A00002808002020000020AE
:10467000446F6E65204269733F000000252520527B
:1046800065706F6E7365206861726D6F6E697175AC
:10469000652E200A46203D205B25322E3266000022
:1046A000846200082C2025322E3266005D3B200AF1
:1046B0004761696E203D205B252E326600000000B8
:1046C000E86200085068617365203D205B252E324A
:1046D00066000000FC630008BC630008616E616C4A
:1046E000797365206861726D2E00000080000020E3
:1046F000D0620008EF620008C86300085463000835
:1047000045020008652A0008FC6200082C630008C6
:10471000BC040020C2620008BD620008A06300085B
:10472000AC62000890630008B06300086D480008A0
:1047300014000020794900081CB500204FF4004106
:1047400000228DF806004020FEF738FF104C01A92A
:10475000FEF7FAFE94F85D000228FBD0FEF7FFFD9D
:104760001CBD00BF1CB58DF806004FF414604FF45B
:1047700000410022FEF722FF054C01A9FEF7E4FEEE
:1047800094F85D000228FBD0FEF7E9FD1CBD00BFD8
:104790002C07002010B5812898BF3F2900D910BDF3
:1047A00001F00703C908012441EA8111012A04FA32
:1047B00003F300EB41003A490A5C14BF9A431A43E1
:1047C0000A5410BD0028364A18BF4FF0FF300021B0
:1047D000B1F5826F08BF704750540131F8E700BF50
:1047E000B0B56420FCF710FF2E4CAE20A04720206F
:1047F000A0471020A047B020A047C820A047002015
:104800000025A0471020A0474020A0478120A047B6
:10481000FF20A047A120A047A620A047A820A0478E
:104820003F20A047A420A047D320A0470020A047B6
:10483000D520A047F020A047D920A0472220A0479C
:10484000DA20A0471220A047DB20A0472020A04765
:104850008D20A0471420A047AF20A0470020FFF7DD
:10486000B1FF00F007F832480560B0BD304A518012
:104870001080704770B50A4C0A4E0025082D08BFFD
:1048800070BDA5F15000C0B2B0470020B047102065
:10489000B0472046822100F05FF882340135EDE711
:1048A000AC000020354900082DE9FE4F204F029250
:1048B0003A8852FA81F2812A04D87A8852FA91F21F
:1048C0003F2A02D90020BDE8FE8F0090C1F3072BDC
:1048D00020381D46CCB2B3FA83F64FF000080BFB2C
:1048E00000F00190D8451CD0019802994FF0000AC1
:1048F000404431F81090544510D009FA0AF02A4685
:10490000000458BF72097988388841445044C9B2BC
:10491000C0B2FFF73FFF0AF1010AECE708F1010816
:10492000E0E73888204438800098BDE8FE8F00BF5B
:1049300078000020F8B58DF80F004FF0FF3001210E
:104940000DF10F02012302900A48CDE900217821E0
:104950000022FCF7DBFF8FBDF8B54FF0FF3289B2C4
:104960008DE807000348012378214022FCF7CEFFA1
:104970008FBD00BFE0060020F8B51C4615460E4668
:104980000746387858B131462A462346FFF78CFF50
:10499000014617F8010B814218BFF8BDF1E700206E
:1049A000F8BD00000FB4084B10B504A902AA039883
:1049B00000F0EAFC044602A9002001F07CF8204641
:1049C00010BC5DF814FB0000B75A00084100080253
:1049D00018BF04200A0E18BF40F001004FF07F42BC
:1049E00032EA010108BF40F00200012808BF05209B
:1049F0007047000070B54FF068422DED048BF0EE6B
:104A0000408A18EE900AB0EE608A18EE101A02EB97
:104A10004003B3F1654F3CBF02EB4102B2F1654F79
:104A20007DD200BFC0F3C753C1F3C7529A1A1B2AE5
:104A300009DD10F0004F14BF9FED830A9FED830A3C
:104A4000BDEC048B70BD12F11A0F36DA11F0004F75
:104A500009D010F0004F0CBF9FED7D0A9FED7D0A3D
:104A6000BDEC048B70BD88EE889A19EE100AFFF732
:104A7000ADFF042808BF00F0FDFA18EE900AFFF71A
:104A8000A5FF054618EE100AFFF7A0FF044619EE31
:104A9000100AFFF79BFF042D18BF052D08D1042C29
:104AA00018BF052C04D1002804BF022000F0A4FB8D
:104AB000B0EE490ABDEC048B70BD4200B2EB410F71
:104AC0003AD910F0004F19BFDFED630A9FED630A7A
:104AD000DFED630A9FED630AB0EE481A0A46B1EEB5
:104AE000688A80F00041F0EE418A10460A1A5200AE
:104AF000B2F1807F34D2484010F0004FDFED5A1AF7
:104B00009FED5A2A1DBFBEEE001A70EEE10A30EE8C
:104B1000420AB6EE001A08BF70EEA10A00E040E0BB
:104B200008BF30EE020AB0EE682A01EE482A08EE0D
:104B3000818AC2EE081A15E011F0004F04BF9FED04
:104B40004C0AF0EE400AD1D010F0004F19BFDFED53
:104B5000490A9FED490ADFED490A9FED490AC5E779
:104B6000C8EE881A21EEA11A9FED462ADFED462AEB
:104B700041EE022A9FED452A01EE222ADFED442A6A
:104B800041EE022A9FED432ABDEC048B01EE222A5E
:104B900021EE811A01EE020A30EE210A30EE200ADF
:104BA00070BD4FF07F42B2EB400F28BFB2EB410F18
:104BB00009D2F0EE480AB0EE680ABDEC048BBDE8FD
:104BC000704000F04BBA40EA01035B0008BF41F0BF
:104BD000FF410BD0B2EB400F08BFB2EB410F08D141
:104BE00020F0804008EE900A21F0804108EE101A73
:104BF00018E7B2EB400F12BF5FEA410340F0FF40FD
:104C000001F000413FF40EAFB2EB410F12BF5FEA7B
:104C1000400200F0004041F0FF413FF403AF4A0082
:104C200092EA40033FF5FEAE002AACBF9FED1A0AA0
:104C30009FED1A0A68EE808A28EE008A18EE900A24
:104C400018EE101AEEE60000DB0FC9BFDB0FC93FFC
:104C5000DB0F4940DB0F49C00000C9BF22AAFDB9E4
:104C60000000C93F22AAFD390060ED3EC30ACE37DD
:104C700000000000000049C022AA7DBA000049409F
:104C800022AA7D3A2DAD65BD8FB8D53D0FB511BEB9
:104C900061C84C3EA8AAAABE0000804F0000802F29
:104CA00010EE101A08B5444A6846B2EB410F28D9F5
:104CB0004FF0E640B0EB410F94BF00204FF0FF30C3
:104CC00000900098002861DB60EE000A10F0010FF0
:104CD00045D010F0020FDFED391A9FED391A00EEC2
:104CE000A11ADFED381A40EE811A21EEA01AF0EE7B
:104CF000400A40EE010A08BFF1EE600AB0EE600A19
:104D000008BD314B21F0004293423CD911F0004FD5
:104D1000DFED2E0A20EE201ADFED2D0A19BF31EE4D
:104D2000601A71EE200A31EE201A71EE600ABDEEB3
:104D3000E01A11EE100A9FED271A00F0030000EEB2
:104D4000C10A9FED251A009000EEC10A9FED231ABB
:104D500000EEC10A9FED221A00EEC10AB1E79FEDF5
:104D6000211A9FED210A10F0020F00EE810A9FED3B
:104D70001F1A00EE801AB7EE000A00EE810A18BF73
:104D8000B1EE400A08BD00F07DF99AE710EE100A76
:104D90004000B0F17F4F3CBFB7EE000A08BD07D11D
:104DA0004FF0010000F028FABDE8084000F05AB9C1
:104DB000BDE8084000F04FB9B61F927E336D4CB984
:104DC000DA82083CA0AA2ABE490E494683F9223F4E
:104DD0000000004B0000C93F00A0FD390020A233B5
:104DE0001A61342CB93AB2BACA9F2A3DDDFFFFBE20
:104DF00010B52DED028BB0EE408A18EE100AFBF7CD
:104E0000D8FB01EE100A18EE100AB7EE000A78EE91
:104E1000410A10F0004F4FF07F4010EE901A12D070
:104E2000B1F13F4F24BF10EE901AB0EB410F12D2F8
:104E300010EE901AB1F17C5F1CDD10EE901AB0EB11
:104E4000410F17D314E0B1F13F4F07D910EE901A7C
:104E5000B0EB410F02D331EE401A0BE010EE901A86
:104E6000B1F17C5F06DB10EE901AB0EB410F01D37D
:104E700031EE001A18EE100ABDEC028B11EE101A7A
:104E800061F31E0000EE100A10BD000000B510EE28
:104E9000101A2DED028B81B0524A6846B2EB410FD9
:104EA0002ED94FF0E640B0EB410F94BF00204FF0F9
:104EB000FF3000900098B0EE408A00286ADB10F0C6
:104EC000010F4BD068EE080A9FED471A9FED470A85
:104ED00000EE810A9FED461A10F0020F00EE801AD4
:104EE000B7EE000A00EE810A02BF01B0BDEC028BF2
:104EF00000BD00BF01B0B1EE400ABDEC028B00BDA9
:104F00003C4B21F00042934241D911F0004FDFEDBC
:104F10003A0A20EE201ADFED390A19BF31EE601A85
:104F200071EE200A31EE201A71EE600ABDEEE01A31
:104F300011EE100A9FED321A00F0030000EEC10AD4
:104F40009FED301A009000EEC10A9FED2F1A00EE7F
:104F5000C10A9FED2E1A00EEC10AABE728EE080A3F
:104F60009FED2B1ADFED2B0A10F0020F40EE010A25
:104F70009FED291A00EE201A61EE000AB0EE480AF1
:104F800008EE200AB6D101B0BDEC028B00BD00F0E6
:104F900079F88FE718EE100A4000B0F17F4F0DD27C
:104FA00018EE100AFFF712FD042808BF00F062F89F
:104FB000B0EE480A01B0BDEC028B00BD09D1012062
:104FC00000F01AF901B0BDEC028B5DF804EB00F0C3
:104FD00049B801B0B0EE480ABDEC028B5DF804EBB5
:104FE00000F039B8B61F927EB93AB2BACA9F2A3DCC
:104FF000DDFFFFBE490E494683F9223F0000004B0A
:105000000000C93F00A0FD390020A2331A61342CF2
:10501000336D4CB9DA82083CA0AA2ABE10B52DED3A
:10502000028BB1EEC08A18EE100A20F00040C0F1E9
:10503000FF40C00F0AD010EE100A20F00040C0F16F
:10504000FF40C00F04BF012000F0D6F8B0EE480AC0
:10505000BDEC028B10BD30EE000A704730EE200A26
:1050600070470000DFED020A80EEA00A70470000E2
:10507000000000009FED020A20EE000A70470000C9
:10508000000000102DE9F0014FF07F42B2EB410F1C
:105090009FBF4FF0FF310160BDE8F00170474FF056
:1050A000004242EA0123C1F3C752783A551112F087
:1050B0001F0C434CCCF120067C44C1F3C752A2F133
:1050C00078024FEA621204EB820254F8254008BFCE
:1050D000D2E9015612D0556804FA0CF425FA06F705
:1050E0003C43976805FA0CF527FA06F8D26807FAE8
:1050F0000CFCF24045EA08054CEA0206A4FB034C0E
:10510000A5FB0352A6FB03631D449D4234BF012649
:1051100000261319334416B1934202D903E0934297
:1051200001D2012200E00022624402F1200C92062A
:10513000DC0C42EA443200EE102A5B03DFED210A68
:10514000F8EEC01A00EE103A4FEA9C1C11F0004F26
:10515000B8EE400AC0F800C020EE201A00EE105A47
:10516000DFED190AB8EE400A20EE200A71EE810A3E
:1051700070EE800A10EE902A02F500626FF30B02C7
:1051800000EE902A70EEE11A31EEC11ADFED101A2E
:1051900030EE411A9FED0D0A20EE800A01EE210A41
:1051A0009FED0C1A00EE810A04BFBDE8F0017047C4
:1051B000CCF180510160BDE8F001B1EE400A7047CA
:1051C000040A0000000000360000802C22AAFD29FD
:1051D000DB0FC92F0000C92F02E008C8121F08C149
:1051E000002AFAD170477047002001E001C1121F68
:1051F000002AFBD170470000014908607047000099
:10520000000000202DE9FF5F82B00021DDE90430BD
:10521000020DDDF840B0034318D044F61050A2F25E
:10522000FF3242431514119801281FD0A5EB0B0043
:10523000401C5FEA000A4FF000064E4FDFF838913D
:10524000B046504615D5CAF1000413E01198012468
:105250004AA3012801D16FEA0B010298119AC0E913
:105260000031C0E9024206B0BDE8F09FCBF100007A
:10527000DFE704460021404A491842EB0450CDE9DB
:10528000001012E0E00707D032463B464046494650
:10529000FBF70AFA8046894632463B4610461946D5
:1052A000FBF702FA06460F466410002CEAD1DDE94E
:1052B0000401DDE90023BAF1000F06DAFBF7F4F987
:1052C00042464B46FBF7F0F905E0FBF769F842462A
:1052D0004B46FBF765F804460E460022284BFBF7C9
:1052E0006DFA03D84FF0FF30014607E00022254B4E
:1052F00020463146FAF7ADFFFBF748FA102409E0E3
:10530000002C0ADB0A220023FBF701F9039B303251
:105310001A55641E50EA0102F2D1641C039AC4F1CA
:1053200011031444119A012A03D0012208430DD11C
:105330000AE0084304D000204FF0110B119072E7EF
:10534000A3EB0B056D1E0DE05B4504DD4FF0000285
:1053500005F1010504E003DA4FF00002A5F10105B3
:10536000002AECD002981199C0E90231C0E9004549
:1053700079E70000000014400000F03F300000001A
:105380000000F0430000E03F2DE9FF4F95B09B4641
:105390008946064600250FE2252877D100242746B6
:1053A000F84A0121059400E0044316F8013F203B30
:1053B00001FA03F01042F7D130782A2811D06FF0AB
:1053C0002F033078A0F13002092A16D8059A44F04C
:1053D000020402EB820203EB42021044761C0590A9
:1053E000EFE759F8042B0592002A03DA504244F4FF
:1053F0000054059044F00204761C30782E2816D113
:1054000016F8010F44F004042A280DD06FF02F0283
:105410003078A0F13003092B09D807EB870302EBA2
:105420004303C718761CF3E759F8047B761C3078E1
:105430006C280FD006DC4C2817D068280DD06A28BD
:1054400014D104E0742810D07A280FD10DE044F470
:1054500000140AE044F4801401E044F4401472782B
:10546000824202D104F58014761C761C30786628BE
:105470000BD013DC582877D009DC002875D04528DC
:10548000F6D04628F4D047281AD19DE118E06328C9
:1054900035D0642879D0652812D195E1702873D071
:1054A00008DC6728F1D069286FD06E280DD06F28EE
:1054B00006D1B5E073282CD0752875D0782874D023
:1054C0005A46179990476D1C75E1C4F302500228A3
:1054D00009D003280DD0D9F8001004280DD00D6094
:1054E00009F1040967E1D9F80010EA17C1E900528F
:1054F000F6E7D9F800100D80F2E70D70F0E719F823
:10550000041B8DF8001000208DF80100EA460120F0
:1055100003E059F804AB4FF0FF3061074FF0000192
:1055200002D40DE008F101018846B9420FDA804546
:10553000F8DB1AF808100029F4D108E008F101019D
:1055400088468142FADB1AF808100029F6D105983E
:105550005B46A0EB080721463846179A00F094FAFC
:10556000284400EB080507E04DE029E10DE01AF8BA
:10557000010B5A4617999047B8F10108F7D25B46DC
:1055800021463846179A13E142E00A220092C4F3FA
:1055900002524FF0000A022A08D059F804CB032A1D
:1055A0004FEAEC710AD00DE029E02AE009F1070189
:1055B00021F00702F2E802C1914609E00FFA8CFCE3
:1055C0004FEAEC71042A03D14FFA8CFC4FEAEC71DC
:1055D000002907DA0A460021DCF1000C61EB020128
:1055E0002D2202E0220504D52B228DF80420012271
:1055F00003E0E20701D02022F7E7904659E00A21B4
:1056000002E010220DE010214FF0000A00910BE0A3
:1056100010224FF0000A44F004040827009203E02F
:1056200008224FF0000A0092C4F30252022A05D069
:1056300059F804CB0021032A08D009E009F1070139
:1056400021F00702F2E802C1914605E01FFA8CFC46
:10565000042A01D10CF0FF0C4FF00008220728D5D6
:10566000702806D0009B83F0100353EA0A0305D08C
:105670000EE040228DF80420012208E05CEA0102DD
:1056800006D030228DF804208DF8050002229046C5
:10569000009B83F0080353EA0A030AD15CEA010283
:1056A00001D1620705D530228DF804204FF00108A2
:1056B0007F1E582804D034A003900EA802900DE05D
:1056C00036A0F9E753466046009AFAF720FF844671
:1056D0000398825C0298401E029002705CEA01000E
:1056E000F0D1029806A9081A00F1200A600702D535
:1056F00024F4803400E00127574502DDA7EB0A00BF
:1057000000E0002000EB0A01009005984144401A97
:105710000590E00306D45B462146179A059800F0F1
:10572000B3F90544002706E001A85A46C05D179961
:1057300090476D1C7F1C4745F6DBE0030CD55B46AC
:105740002146179A059800F09FF9054404E030209F
:105750005A46179990476D1C0099481E00900029E1
:10576000F5DC08E0029802995A460078491C02913B
:10577000179990476D1CBAF10001AAF1010AF1DCFA
:1057800065E1000009280100303132333435363705
:10579000383961626364656600000000303132337D
:1057A000343536373839414243444546000000001D
:1057B00000F058F90544761C307800287FF4ECADF1
:1057C00019B02846BDE8F08F620700D4062709F11A
:1057D000070222F0070CFCE80223E14603F0004830
:1057E0005FEA080C02D00FF2702C0DE05FEA045C57
:1057F00002D50FF2682C07E05FEAC47C02D00FF2FA
:10580000602C01E0AFF2700C4FF0FF3823F0004342
:10581000CDF850C065280CD006DC452809D04628B4
:105820001DD047283DD13DE0662818D067287ED19D
:1058300038E00021112F01DB112000E0781CCDE9B8
:10584000000106A90EA8FFF7DDFCDDE90F010E9AA5
:1058500003910021009207F1010A04914DE04FF0FD
:1058600000400097CDE9011006A90EA8FFF7CAFC79
:10587000DDE90F0203920E9B11990022DDF80CA0C6
:105880000093049211B9791C00EB010AB7EB0A00EE
:1058900004D4C0F1FF3007F1010A0490AAEB07001D
:1058A000019044E0012F00DA01270021112F01DDD2
:1058B000112000E03846CDE9000106A90EA8FFF747
:1058C000A1FCDDE90F010E9A0391002104910092E1
:1058D000BA4621070CD40399514500DA8A46BAF139
:1058E000010F05DD009AAAF10101515C302908D0B1
:1058F000B84202DA10F1040F06DA0121CDE90110F5
:1059000015E0AAF10101E9E7002805DC049901444A
:105910000491AAEB000102E0411C514500DD8A46DA
:105920000499401A401C01904FF00040029020075B
:1059300004D40198504501DBCDF8048000208DF897
:105940004F0002980DF14F07B0F1004F25D02B20EA
:105950000E9002984FF0020800280CDA40420290A4
:105960002D200E9007E00A210298FAF7BAFD303197
:10597000029007F8011DB8F10001A8F10108F2DC5E
:1059800002980028EFD1791E0E980870307800F048
:10599000200040F0450007F8020D12A8C01B00F1DE
:1059A00007081498007800B1012000EB0A01019863
:1059B00001EBE07105984144401A401E0590E00358
:1059C00006D45B462146179A059800F05DF8054419
:1059D0001498007818B15A46179990476D1CE00347
:1059E00024D55B462146179A059800F04DF80544EA
:1059F0001CE00498002807DBDDE90301884203DD91
:105A00000098405C179901E0179930205A4690475A
:105A1000049805F10105401C04900198401E019076
:105A200004D12E205A46179990476D1CBAF10001F7
:105A3000AAF1010ADDDC05E017F8010B5A461799B7
:105A400090476D1CB8F10001A8F10108F4DC5B4639
:105A50002146179A0598ABE62D0000002B000000A8
:105A6000200000002DE9F041044600251E4617469F
:105A7000880404D405E039462020B0476D1C641E1C
:105A8000F9D52846BDE8F0812DE9F041044600250E
:105A90001E469046C80301D5302700E02027880421
:105AA00004D505E041463846B0476D1C641EF9D563
:105AB0002846BDE8F0810A68531C0B6010707047DF
:105AC000000000006E83F9A22915444ED15727FC2F
:105AD000C0DD34F5999562DB4190433CAB6351FEE8
:105AE000000000000000000001020304060708098E
:105AF000000000000102030400000000000000009C
:105B00000000000000000000000000000010001075
:105B10000010001000100010000000100000000035
:105B200000280028002800000000000000000000FD
:105B30000000000000240024007C00240048007CB9
:105B400000480048000000000038005400500038B1
:105B500000140054005400380010000000200054CD
:105B60000058003000280054001400080000000015
:105B700000100028002800100034004800480034BD
:105B800000000000001000100010000000000000E5
:105B900000000000000000000008001000200020AD
:105BA000002000200020002000100008002000102D
:105BB0000008000800080008000800080010002085
:105BC0000010003800100028000000000000000055
:105BD000000000000000000000100010007C001019
:105BE00000100000000000000000000000000000A5
:105BF0000000000000000010001000100000000075
:105C0000000000000000003800000000000000005C
:105C10000000000000000000000000000000001074
:105C20000000000000080008001000100010001024
:105C30000020002000000000003800440044005410
:105C40000044004400440038000000000010003010
:105C500000500010001000100010001000000000A4
:105C60000038004400440004000800100020007CBC
:105C70000000000000380044000400180004000484
:105C80000044003800000000000800180028002828
:105C90000048007C0008000800000000007C004074
:105CA00000400078000400040044003800000000B8
:105CB00000380044004000780044004400440038AC
:105CC00000000000007C000400080010001000200C
:105CD000002000200000000000380044004400388C
:105CE0000044004400440038000000000038004434
:105CF00000440044003C0004004400380000000060
:105D00000000000000100000000000000000001073
:105D10000000000000000000000000100000000073
:105D2000000000100010001000000000000C003007
:105D300000400030000C00000000000000000000E7
:105D40000000007C0000007C00000000000000005B
:105D5000000000000060001800040018006000004F
:105D6000000000000038004400040008001000108B
:105D7000000000100000000000380044004C0054F7
:105D8000005C0040004000380000000000100028C7
:105D9000002800280028007C004400440000000087
:105DA0000078004400440078004400440044007837
:105DB0000000000000380044004000400040004067
:105DC0000044003800000000007000480044004417
:105DD000004400440048007000000000007C0040C7
:105DE0000040007C004000400040007C00000000BB
:105DF000007C00400040007800400040004000402F
:105E0000000000000038004400400040005C0044F6
:105E10000044003800000000004400440044007CBE
:105E2000004400440044004400000000003800101A
:105E300000100010001000100010003800000000DA
:105E400000040004000400040004000400440038BE
:105E5000000000000044004800500060005000486E
:105E600000480044000000000040004000400040A6
:105E7000004000400040007C000000000044006C36
:105E8000006C005400440044004400440000000042
:105E900000440064006400540054004C004C004472
:105EA0000000000000380044004400440044004466
:105EB0000044003800000000007800440044004422
:105EC000007800400040004000000000003800441E
:105ED0000044004400440044005400380004000022
:105EE0000078004400440044007800480048004422
:105EF00000000000003800440040003000080004AA
:105F00000044003800000000007C00100010001069
:105F100000100010001000100000000000440044B9
:105F200000440044004400440044003800000000E5
:105F300000440044004400280028002800100010FD
:105F40000000000000440044005400540054006C61
:105F5000002800280000000000440028002800104D
:105F60000010002800280044000000000044004405
:105F70000028002800100010001000100000000091
:105F8000007C000400080010001000200040007C8D
:105F90000000000000180010001000100010001099
:105FA0000010001000100018002000200010001049
:105FB0000010001000080008000000000030001071
:105FC0000010001000100010001000100010003031
:105FD000001000280028004400000000000000001D
:105FE00000000000000000000000000000000000B1
:105FF00000000000000000FE002000100000000073
:106000000000000000000000000000000000000090
:1060100000380044003C0044004C00340000000004
:1060200000400040005800640044004400640058F0
:106030000000000000000000003800440040004064
:106040000044003800000000000400040034004C4C
:1060500000440044004C0034000000000000000038
:1060600000380044007C004000440038000000007C
:10607000000C0010007C0010001000100010001038
:1060800000000000000000000034004C0044004408
:10609000004C0034000400780040004000580064C8
:1060A00000440044004400440000000000100000D0
:1060B0000070001000100010001000100000000020
:1060C0000010000000700010001000100010001000
:1060D000001000E000400040004800500060005008
:1060E0000048004400000000007000100010001084
:1060F0000010001000100010000000000000000060
:106100000078005400540054005400540000000073
:1061100000000000005800640044004400440044B3
:10612000000000000000000000380044004400446B
:106130000044003800000000000000000058006427
:10614000004400440064005800400040000000008B
:106150000034004C00440044004C003400040004AF
:106160000000000000580064004000400040004073
:10617000000000000000000000380044003000086B
:1061800000440038000000000020002000780020BB
:106190000020002000200018000000000000000087
:1061A0000044004400440044004C0034000000005F
:1061B00000000000004400440028002800280010CF
:1061C0000000000000000000005400540054006C67
:1061D0000028002800000000000000000044002803
:1061E0000010001000280044000000000000000023
:1061F0000044004400280028001000100010006037
:1062000000000000007C0008001000200040007C1E
:1062100000000000001800100010001000200020F6
:1062200000100010001000180010001000100010E6
:1062300000100010001000100010001000300010BE
:1062400000100010000800080010001000100030BE
:106250000000000000000074004C0000000000007E
:106260000000000002030405060708090A0B0C0DD4
:106270000E0F10100102030405060708090A0B0C93
:106280000D0E0F100000803F4D84D53F1E1632408A
:10629000FD87944061C3F740E3A54E41BA5AAC4133
:1062A0009DC00F4229CB6F420000C8424370745F0B
:1062B000416371203D202564202E2E2E002C2025A8
:1062C000640056697465737365203D205B25640026
:1062D000663D25322E30662C473D25322E30662C09
:1062E000503D25322E3066002C20252E3266006669
:1062F000203D2025322E3266000000002520526508
:10630000706F6E736520696E64696369656C6C6536
:106310002064652072203D203230252061207220CB
:106320003D2031303025200A000000002520506536
:1063300072696F6465206427656368616E74696C57
:106340006C6F6E6E616765205465203D20316D7302
:106350000A00000025204964656E746966696361FE
:1063600074696F6E2074656D706F72656C6C6520FA
:106370000A2D2D2D2D2D2D2D2D2D2D2D2D2D2D2D70
:106380002D2D2D2D2D2D2D2D2D2D2D2D20000000D1
:1063900042505F5550203D3D3E20313030250000B9
:1063A00050574D3D31303025202E2E2E000000005C
:1063B00050574D3D323025202E2E2E0050574D3D4A
:1063C000363025202E2E2E00446F6E652E20426919
:1063D000733F000042505F555020322A2049642EFE
:1063E0002074656D7000000042505F555020322AC5
:1063F0002049642E206672657100000042505F449F
:106400004F574E20706F7572000000003064000816
:106410000000002020000000D8510008506400084F
:1064200020000020900E0000E8510008000000004D
:10643000000000000000803F0000803F01000000DD
:1064400010000000070A0000F85A000800127A0045
:040000050800018965
:00000001FF
